:100000000C941E0B0C94460B0C94460B0C94460B54
:100010000C94460B0C94460B0C94460B0C94460B1C
:100020000C94460B0C94460B0C94460B0C94460B0C
:100030000C94460B0C94460B0C94460B0C94460BFC
:100040000C9484160C94460B0C94460B0C94460BA3
:100050000C94460B0C94460B0C94460B0C94460BDC
:100060000C94CE160C94460BFFE0FFD1AFFF32FF8D
:10007000D0FFFEFFE0FFD1AEFFD0FFFEFFE0FFD1DB
:100080001000FFFEFFD0FFE0FFC1FFD1AED580A87A
:100090003FD300408D142000A1C8DA1281CFD9F1DE
:1000A000DB402EA4A6AFFFD0FFFE0000000025001D
:1000B00028002B00000000080002010000030407D4
:1000C00000000000000000000000000024002700E5
:1000D0002A00FFFFFFFFFFFFFFFFFFFFFFFFFFFF04
:1000E000FFFF010000000000000000000000000011
:1000F000008001000000000000000000000000007F
:10010000008001000000000000000000000000006E
:10011000008001000000000000000000000000F06E
:10012000FFBF010000000000000000000000001000
:1001300000A0010000000000000000000000001C02
:1001400000A0010000000000000000000000001CF2
:1001500000A0010000000000000000000000001CE2
:1001600000A0010000000000000000000000001CD2
:1001700000A0010000000000000000000000001CC2
:1001800000A00100000000000000000000000010BE
:1001900000A001000000000000000000000000F0CE
:1001A000FFBF010000000000000000000000000090
:1001B00000800100000000000000000000000000BE
:1001C0000080FFFFFFFFFFFFFFFFFFFFFFFFFFFFBD
:1001D000FFFF010000000000000000000000000020
:1001E000008001000000000000000000000000008E
:1001F000008001000000000000000000000000007E
:10020000008001000000000000000000000000006D
:10021000008001000000000000000000000000005D
:10022000008001000000000000000000000000004D
:10023000008001000000000000000000000000003D
:10024000008001000000000000000000000000002D
:10025000008001000000000000000000000000001D
:10026000008001000000000000000000000000000D
:1002700000800100000000000000000000000000FD
:1002800000800100000000000000000000000000ED
:1002900000800100000000000000000000000000DD
:1002A00000800100000000000000000000000000CD
:1002B00000800100000000000000000000000000BD
:1002C00000800100000000000000000000000000AD
:1002D000008001000000000000000000000000009D
:1002E000008001000000000000000000000000008D
:1002F000008001000000000000000000000000007D
:10030000008001000000000000000000000000006C
:10031000008001000000000000000000000000005C
:10032000008001000000000000000000000000004C
:10033000008001000000000000000000000000003C
:10034000008001000000000000000000000000002C
:10035000008001000000000000000000000000001C
:10036000008001000000000000000000000000000C
:1003700000800100000000000000000000000000FC
:1003800000800100000000000000000000000000EC
:1003900000800100000000000000000000000000DC
:1003A00000800100000000000000000000000000CC
:1003B00000800100000000000000000000000000BC
:1003C00000800100000000000000000000000000AC
:1003D000008001000000000000000000000000009C
:1003E000008001000000000000000000000000008C
:1003F000008001000000000000000000000000007C
:10040000008001000000000000000000000000006B
:10041000008001000000000000000000000000005B
:10042000008001000000000000000000000000004B
:10043000008001000000000000000000000000003B
:10044000008001000000000000000000000000002B
:10045000008001000000000000000000000000001B
:10046000008001000000000000000000000000000B
:1004700000800100000000000000000000000000FB
:1004800000800100000000000000000000000000EB
:1004900000800100000000000000000000000000DB
:1004A00000800100000000000000000000000000CB
:1004B0000080FFFFFFFFFFFFFFFFFFFFFFFFFFFFCA
:1004C000FFFFFFFFFFFFFFFFFFFFFFFFFFFFFFFF3C
:1004D000FFFF00000000230026002900040404049C
:1004E00004040404020202020202030303030303DE
:1004F00001020408102040800102040810200102BB
:1005000004081020000C11FEFC0701930338207F23
:10051000FE08FD07FE0000000200010107070301BD
:100520000080808080800080030202040005A0A07B
:100530000507070500005050F850F850500409090D
:100540000500FF20709080601090E02007070708EA
:1005500000007EA4A8562A2A440807070800003095
:10056000506E74988D7601020202000580800309A6
:10057000090400FE2040408080804040200309099B
:100580000400FE80404020202040408003030305FB
:100590000104A040A00505050600002020F8202049
:1005A0000202020300FFC040030101040002E00157
:1005B00001010301008003070703000020204040E1
:1005C0004080800407070500006090909090906044
:1005D00003070705010040C040404040E004070712
:1005E000050000609010202040F00407070500007F
:1005F000609010601010E0050707050000103050F3
:1006000090F810100407070500007040E01010106B
:10061000E00407070500003040E090909060040778
:1006200007050000F0902020404040040707050027
:100630000060909060909060040707050000609053
:1006400090907020C001050503010080000000802B
:100650000206060300FF40000000C0400305050538
:1006600001002040804020050303060001F800F847
:1006700003050505000080402040800307070400B3
:1006800000E0A020404000400809090900FE3C426B
:100690009DA5A5AD92403E07070708000010382829
:1006A000287C44EE050707060000F04848704848DB
:1006B000F00607070700007CC4808080C478060726
:1006C00007070000F84C4444444CF80507070600AF
:1006D00000F84840704048F8050707060000F84851
:1006E00040704040E00607070700007CC4809C84FF
:1006F000C478070707080000EE44447C4444EE0336
:100700000707040000E04040404040E004070704C1
:1007100000007020202020A0C0060707070000EC82
:100720004850605048EC050707060000E040404094
:100730004048F809070E0A0000E3806300550055A1
:10074000005D004900EB80070707080000EE6454D5
:10075000544C4CE406070707000078CC848484CC12
:1007600078050707060000F04848704040E0060999
:10077000090700FE78CC848484CC70180C06070727
:10078000070000F04848705048EC040707050000D7
:100790007090C0601090E0050707060000F8A820E0
:1007A00020202070070707080000EE444444446CF2
:1007B00038070707080000EE446C282810100B07C4
:1007C0000E0AFF00EEE0444064C02E802A80110033
:1007D0001100070707080000EE4428102844EE0720
:1007E0000707080000EE44283810103805070706F0
:1007F0000000F88810204088F80209090300FEC0B4
:1008000080808080808080C0030707030000808094
:1008100040404020200209090300FEC04040404003
:10082000404040C003030305010440A0A0050101AE
:100830000500FDF8020202030006804003050504DE
:100840000000C02060A0E005070705FF00C0407061
:1008500048484870030505040000608080806005FA
:10086000070705000030107090909068030505049C
:10087000000060A0C080600407070400003040E072
:10088000404040E00407070500FE70A0A0406090D3
:10089000E006070705FF00C040704848486C0207A3
:1008A000070300004000C04040404003090903FF27
:1008B000FE2000602020202020C006070705FF0042
:1008C000C040485070484C030707040000C0404037
:1008D000404040E0080505080000EC929292DB05DC
:1008E0000505050000E0909090D80405050500007E
:1008F000609090906005080805FFFDF0484848703A
:100900004040E00508080500FD70909090701010C0
:1009100038030505040000A0604040E0030505041D
:10092000000060804020E004060604000040E04033
:10093000404030050505050000D8909090680605F8
:100940000505FF00EC4828301009050A08FF00EDF6
:100950008049002A0036001400050505060000D86D
:10096000502050D806070705FFFEDC4850302060B5
:10097000C0040505050000F0204090F003090904BB
:1009800000FE204040408040404020010909020014
:10099000FE8080808080808080800309090400FEC2
:1009A0008040404020404040800602020700026430
:1009B00098FF001D25FCF711040908F1207FFA13A8
:1009C000FA11FA00000006000103111108030040AB
:1009D000E0E0E0E0E0E0E040404040000000C0C077
:1009E0000605050A010CCCCCCCCC880B11220D01DC
:1009F00000088008800880088008807FE07FE01180
:100A00000011001100FFC0FFC022002200220022BE
:100A10000022000B152A0C00FE040004003F0065B4
:100A2000C0C4C0C440C440E4007C001E0007800570
:100A3000C004E0046084608460C4C0E5C03F00047A
:100A40000004001110301301001E0C0033FC006183
:100A50001800C11000C13000C26000E4400078C03E
:100A600000018F00011980033080066080046080DF
:100A70000C6100187200103C0011113313010007C3
:100A8000C0000860001820001820001860000CC08A
:100A9000000F9E00070C000F0800338800619000D3
:100AA000C0D000C0E000C06000E0F0807FBF003E2A
:100AB0000E0002050506020CC0C0C0C08006161656
:100AC0000801FB04081030206060C0C0C0C0C0C076
:100AD000C0C0606020301008040616160801FB80B4
:100AE0004020301018180C0C0C0C0C0C0C0C1818A6
:100AF00010302040800909120C02081C001C00C99B
:100B000080EB801C00EB80C9801C001C000C0C18C2
:100B10000C000006000600060006000600FFF0FFBD
:100B2000F0060006000600060006000305050702A1
:100B3000FDC0E02060C0060202080005FCFC0202C5
:100B400002060200C0C009152A07FEFC01800180D0
:100B500001000300030002000600060004000C0070
:100B60000C00080018001800100030003000600071
:100B700060004000C0000A11220C01001E0033007A
:100B800061806180C0C0C0C0C0C0C0C0C0C0C0C0A3
:100B9000C0C0C0C0E1C06180618033001E00081188
:100BA000110C0200081878181818181818181818B6
:100BB00018181818FF0A11220C01001C007F0043AE
:100BC0008081808180018001800300030006000491
:100BD000000C00180030006040FFC0FF80091122A7
:100BE0000C01001C007E0047008300830006000CFF
:100BF000001E00070003800180018001800100C306
:100C000000E60078000A11220C010003000700072B
:100C1000000B001B0013003300230063004300C3DC
:100C200000FFC0FFC003000300030003000A1122FD
:100C30000C01001FC01F8020002000600078007E93
:100C4000000F80038001C000C000C000C000C0C110
:100C500080E3807E000A11220C010003C00E001800
:100C600000300070006000EE00F380C180C0C0C0A2
:100C7000C0C0C0C0C0E0C061807B801E000A1122DD
:100C80000C01007FC0FFC0C0C08180018001000353
:100C900000030002000600060004000C000C000C1B
:100CA00000180018000A11220C01001E0033006118
:100CB000806180618073003E001E003F00638041C0
:100CC000C0C0C0C0C0C0C0E18073801E000A112235
:100CD0000C01001E0077806180C1C0C0C0C0C0C0D0
:100CE000C0C0C061C073C01D8001800380030006C6
:100CF000001C00F000020B0B060200C0C000000048
:100D000000000000C0C0030E0E0702FDC0C00000BE
:100D10000000000000C0E02060C00B0B160E0100B8
:100D2000006001C007001C007000C00070001C00C3
:100D3000070001C0006009050A0D0203FF80FF8063
:100D40000000FF80FF800B0B160D0100C00070003B
:100D50001C00070001C0006001C007001C007000FB
:100D6000C0000811110B02007CC683C3C3070E0C20
:100D70001C181810100000303012143C1602FD032D
:100D8000F8000F0E001C030038018070008060EC3A
:100D9000C0E1FC40C38C40C30C40C60C40C61840A8
:100DA000C618C0C61880C63980637B0061DE00307B
:100DB00000001800000E0C0003F0001111331100A8
:100DC0000000800001C00001C0000160000260005E
:100DD0000230000630000430000418000C18000F28
:100DE000F800080C00180C00100C0010060030066B
:100DF00000FC1F800E1122100100FFC03070303047
:100E0000301830183018303030403FE0303830186B
:100E1000300C300C300C30183078FFE00E112210FE
:100E2000010007E41C3C380C60046004C000C000F2
:100E3000C000C000C000C000C000600060043808EE
:100E40001E3807E00F1122110100FFC0307030384A
:100E5000300C300C300630063006300630063006D6
:100E60003006300C300C30383070FFC00D11220FBE
:100E70000100FFF0303030103010300030003040D2
:100E800030403FC030403040300030003008300843
:100E90003018FFF80C11220E0100FFF03030301036
:100EA000301030003000302030203FE03020302043
:100EB00030003000300030003000FC0010112212F1
:100EC000010007E41C3C380C60046004C000C00052
:100ED000C000C000C03FC00CC00C600C600C381CCF
:100EE0001E3807E0111133130100FC1F803006008B
:100EF00030060030060030060030060030060030B4
:100F000006003FFE003006003006003006003006C6
:100F100000300600300600300600FC1F800611116C
:100F2000080100FC3030303030303030303030307C
:100F3000303030FC0911220B01001F800600060032
:100F40000600060006000600060006000600060071
:100F5000060006000600C600CC0078001011221121
:100F60000100FC7E30183030306030C031803300FA
:100F70003E003F00338031C030E030703038301CEC
:100F8000300EFC1F0D11220E0100FC00300030005D
:100F900030003000300030003000300030003000D1
:100FA00030003000300830083018FFF815113316C3
:100FB0000100F000F83000E03801603801602C02D8
:100FC000602C02602602602604602304602308600F
:100FD00021886021886020D06020D060206060205F
:100FE0006060F861F8101122120100F01F3004381F
:100FF0000438042C0426042604230421842184209C
:10100000C4206420642034201C201CF80C10112201
:1010100012010007E01C38381C60066006C003C0DF
:1010200003C003C003C003C003C0036006600638EA
:101030001C1C3807E00D11220F0100FFC03070307A
:1010400030301830183018303030703FC030003039
:101050000030003000300030003000FC0010162C52
:101060001201FB07E01C38381C60066006C003C094
:1010700003C003C003C003C003C00360066006389A
:101080001C1C3807E001C000E000700038000F0FA2
:101090001122100100FFC03070303030183018308D
:1010A00018303030703FC03380318030C030603015
:1010B000703038301CFC1E0B11220D01001E4063E5
:1010C000C0C0C0C040C040E00078001E000F8003D8
:1010D000C000E0006080608060C0C0F1809E000EB3
:1010E0001122100100FFFCC30C83048304030003DE
:1010F00000030003000300030003000300030003D8
:1011000000030003000FC0101122120100FC1F3069
:10111000043004300430043004300430043004302F
:1011200004300430043004300818081C3007E01183
:101130001133110000FC1F80300600300400180C31
:10114000001808001808000C18000C1000063000E9
:1011500006200006200003600003400003C00001D9
:101160008000018000018000171133170000FC7E11
:101170007E301818301810181810181830182C2035
:101180000C2C200C2C60064C60064C40064640039C
:1011900046C003468003878001838001830001836A
:1011A000001211331200007E0F801C06000E0C008E
:1011B00006080003100001A00001C00000C00000EC
:1011C000E000017000023800061800040C00080E50
:1011D00000180700300380FC0FC01011221201001C
:1011E000FC3F300C380818181C100C300620066024
:1011F000034003C0018001800180018001800180E3
:1012000007E00D11220F0100FFF0C07080E080C0E8
:1012100001C003800300070006000E001C00180038
:10122000380030087008E018FFF80515150802FCB2
:10123000F8C0C0C0C0C0C0C0C0C0C0C0C0C0C0C076
:10124000C0C0C0C0F8071111070000C0C0406060F6
:10125000203030101818080C0C0406060515150867
:1012600001FCF81818181818181818181818181851
:10127000181818181818F80909120B010808001C8A
:101280000014003600220063004100C18080800C01
:1012900002040C00FBFFF0FFF005040408010DC080
:1012A000E07018090C180B01003E00670063000392
:1012B000000F003B006300C300C300C700FB0071C8
:1012C000800B11220C00003000F0003000300030A4
:1012D00000370039C030C03060306030603060307E
:1012E00060306030C039C02F00090C180B01001F9E
:1012F0000063804180C000C000C000C000C000E0AA
:101300000070807F001E000A11220C01000180077E
:10131000800180018001801D8073806180C180C157
:1013200080C180C180C180C18063807F8019C00975
:101330000C180B01001E0063004180C180FF80C0BB
:1013400000C000C000E00070807F001E0007111187
:101350000700000E16303030FE3030303030303084
:10136000303030780B12240C01FA1EC023C061000B
:10137000618061806180618033003C0040006000DA
:101380007F803FC040E0C060C060E1C07F000C11C2
:10139000220D00003000F0003000300030003380BB
:1013A00037C038E0306030603060306030603060CE
:1013B0003060306078F004111106010060600000B8
:1013C0000060E0606060606060606060F006171759
:1013D00006FEFA0C0C0000000C1C0C0C0C0C0C0C87
:1013E0000C0C0C0C0C0C0CCCC8700C11220C00005A
:1013F0003000F00030003000300033E03180330046
:10140000320034003C0036003700338031C030E019
:1014100079F005111106000030F0303030303030F6
:10142000303030303030303078120C241401006706
:101430000E00EF9F0071E38060C18060C18060C1D9
:101440008060C18060C18060C18060C18060C180F7
:10145000F1E3C00B0C180D01006700EF8071C06054
:10146000C060C060C060C060C060C060C060C0F1EB
:10147000E00A0C180C01001E0073806180C0C0C01F
:10148000C0C0C0C0C0C0C0C0C0618073801E000AA0
:1014900012240C01FA6E00F380618060C060C060AD
:1014A000C060C060C060C0618073806E006000601A
:1014B00000600060006000F0000A12240C01FA1DB8
:1014C0008073806180C180C180C180C180C180C1C2
:1014D00080618073801D8001800180018001800116
:1014E0008003C0060C0C0801006CEC70606060604A
:1014F00060606060F0080C0C0A01003E46C2E070BB
:101500007C1E070383C6F8070F0F0700001030701A
:10151000FE303030303030303030321C0B0C180D93
:101520000100E1C060C060C060C060C060C060C059
:1015300060C060C071C03EC01CE00B0C180B000006
:10154000F1E060C060803080308031001900190007
:101550001A000E000E000400110C24110000F1E727
:101560008060C30060C20030C20030C2003164003D
:101570001964001A64001A28000E38000E3800049E
:1015800010000B0C180D0100F1E060C03180390033
:101590001A000C000E001B003380218060C0F1E0B7
:1015A0000C12240BFFFA78F03060304018401840DD
:1015B00018800C800C800D00070007000200060058
:1015C00004000C00C800F0006000080C0C0A0100C8
:1015D000FFC3860E1C1838307061C3FF0816160A48
:1015E00001FB070C1818181818103020C0203010F4
:1015F0001818181818180C07021111050100C0C09E
:10160000C0C0C0C0C0C0C0C0C0C0C0C0C0C0C00892
:1016100016160A01FBE0301818181818080C0403F5
:10162000040C0818181818181830E00B04080D01DD
:101630000438207C60C7C08380FFE91711241FBED7
:10164000CFEFD8E0DEBFCDBF11E0A0E0B1E0E4E72E
:10165000F7E402C005900D92A238B107D9F723E054
:10166000A2E8B1E001C01D92A034B207E1F71BE08F
:10167000CEE1DBE004C02197FE010E94D320CD31F2
:10168000D107C9F70E9484180C94B8230C94000069
:10169000089580E008958091FC029091FD020097EA
:1016A00039F120910F03FC01211123C03596E491FB
:1016B000E0931003FC013C96E491E09311038091C8
:1016C0001003082E000C990B20911103821B910925
:1016D00027FD939520911203203441F0829FC00191
:1016E000112426E0969587952A95E1F780931303B8
:1016F0000895213039F43F96E491E0931003FC0102
:101700007096DACF3D96E491E0931003FC013E968B
:10171000D3CF8091760290917702891B990B08951F
:10172000AF92BF92CF92DF92EF92FF920F931F93EF
:10173000CF93DF936C017B018B01040F151FEB012D
:101740005E01AE18BF08C017D10759F06991D601E4
:10175000ED91FC910190F081E02DC6010995892B56
:1017600079F7C501DF91CF911F910F91FF90EF9015
:10177000DF90CF90BF90AF90089590E0FC01EC54C3
:10178000FF4F2491FC01E051FB4F3491FC01E452E6
:10179000FB4FE491EE23C9F0222339F0233001F10D
:1017A000A8F4213019F1223029F1F0E0EE0FFF1FEB
:1017B000E655FF4FA591B4918FB7F894EC91611164
:1017C00026C030953E233C938FBF08952730A9F063
:1017D0002830C9F0243049F7809180008F7D03C004
:1017E000809180008F7780938000DFCF84B58F77E2
:1017F00084BDDBCF84B58F7DFBCF8091B0008F7728
:101800008093B000D2CF8091B0008F7DF9CF3E2B76
:10181000DACFCF93DF9390E0FC01E051FB4F2491AE
:1018200084529B4FFC0184918823D1F090E0880F73
:10183000991FFC01E853FF4FA591B491FC01E655B7
:10184000FF4FC591D49161110EC09FB7F8948C9150
:10185000E22FE0958E238C932881E223E8839FBFBB
:10186000DF91CF9108958FB7F894EC91E22BEC9330
:101870008FBFF6CF3FB7F89480914B0290914C0206
:10188000A0914D02B0914E0226B5A89B05C02F3FF6
:1018900019F00196A11DB11D3FBFBA2FA92F982F96
:1018A0008827BC01CD01620F711D811D911D42E091
:1018B000660F771F881F991F4A95D1F708958F9259
:1018C0009F92AF92BF92CF92DF92EF92FF924B0125
:1018D0005C010E943A0C6B017C010E943A0C6C196D
:1018E0007D098E099F09683E734081059105A8F323
:1018F00021E0821A9108A108B10888EEC80E83E0A1
:10190000D81EE11CF11C81149104A104B10429F733
:10191000FF90EF90DF90CF90BF90AF909F908F900F
:101920000895DC011696ED91FC91179712968C9113
:10193000481B477081E090E001C0880F4A95EAF7A4
:10194000E60FF11D3081222319F0832B8083089547
:1019500080958323FBCFFB014181DC0112962C9102
:101960001297421768F013962C911397241740F0A2
:10197000608115962C91621718F424810C94910CB7
:101980000895FC0180819281980F928321819217A2
:1019900060F494819F5F94839381890F821710F084
:1019A0008FEF820F838381E0089580E00895FC012A
:1019B000128280818150838314820895DB01ED912E
:1019C000FC9109940F931F93CF93DF931F92CDB790
:1019D000DEB70091FA021091FB02E0912903F09129
:1019E0002A0382E0099530E020E04AE0B80188EF60
:1019F00092E00E94DE0C182FE0912903F0912A0357
:101A000083E00995E0912903F0912A0380E009958C
:101A10001123B9F16091FA027091FB029E012F5FD0
:101A20003F4F46E488EF92E00E94DE0C898180936C
:101A3000F8026091FA027091FB029E012F5F3F4F06
:101A400047E488EF92E00E94DE0C89818093F902DE
:101A50006091FA027091FB0230E020E048E488EFE8
:101A600092E00E94DE0C809303036091FA02709171
:101A7000FB022BE233E047E188EF92E00E94DE0CAC
:101A800011E0812F0F90DF91CF911F910F91089559
:101A9000CF93DF9380913103811105C081E0809362
:101AA00031030E94E20CC091FA02D091FB02E09156
:101AB0002903F0912A0382E00995E0912903F0912E
:101AC0002A0381E0099530E020E044E1BE0188EF7F
:101AD00092E00E94DE0C2BE233E047E1BE0188EF8A
:101AE00092E00E94DE0CE0912903F0912A0380E04D
:101AF000DF91CF9109941F93CF93DF93182F87E045
:101B000068276F5F6770DFEF01C0DD0F6A95EAF746
:101B1000C6E06091FA027091FB0210931403C09327
:101B2000150310921703D093160324E133E04BE31F
:101B300088EF92E00E94DE0CCF5FCB3051F7DF914F
:101B4000CF911F9108950F931F93CF93E0910603B8
:101B5000F0910703309719F088EF92E00995009112
:101B6000FA021091FB02E0912903F0912A0382E02E
:101B70000995E0912903F0912A0381E0099530E06D
:101B800020E045E1B80188EF92E00E94DE0CC82F0A
:101B9000882341F02BE233E047E1B80188EF92E07F
:101BA0000E94DE0CE0912903F0912A0380E0099560
:101BB0008C2FCF911F910F910895CF92DF92EF92CA
:101BC000FF920F931F93CF93DF93D82FC62FF42E3E
:101BD000042F081B2617D8F4162F121B011708F123
:101BE000812F102F082FD12CE12EE694CC24C39402
:101BF000C21710F0CC24CA94FD16D8F4DF91CF910F
:101C00001F910F91FF90EF90DF90CF900895122FCA
:101C1000161B011728F7F22E242F8D2FD62FC82F31
:101C200005C0C42FF62E8D2FD22F282FDD24D3945C
:101C3000DBCF6091FA027091FB02D11012C0D093F9
:101C40001403C093150324E133E042E388EF92E0EC
:101C50000E94DE0CE01AE7FE02C0CC0DE10EDF5F51
:101C6000CBCFC0931403D0931503EDCF0B96FC019B
:101C7000849108950A96FC0184910895FC01849151
:101C800008950E943E0E882321F0823011F083E0F7
:101C9000089586E00895FC01E60FF11D849190E01F
:101CA000982F88273196E4918E0F911D089568E052
:101CB0000C944B0E66E00C944B0E2EE93FE000971F
:101CC00009F40895F9013197F1F70197F8CFCF930F
:101CD000DF9300D0CDB7DEB720ED37E03A8329831C
:101CE0009091BC00982311F081E00FC029813A81C6
:101CF000232B81F48091750281FDF6CF80917402CF
:101D000081110DC091E0909374020F900F90DF91BC
:101D1000CF91089529813A8121503109DFCF80E0A8
:101D2000F4CF84EA8093BC0061E080E80E94670EF3
:101D3000811102C080E008958091B900887F8830C9
:101D400051F0803141F0809174028111F3CF82E033
:101D500080937402EFCF88E78093BB0084E8809380
:101D6000BC0062E080E80E94670E882319F380912E
:101D7000750281FD05C08091B900887F883119F70F
:101D800081E0089584E98093BC0064E080E10C94D4
:101D9000670E8093BB0084E88093BC0063E080E81A
:101DA0000E94670E8823A1F08091750281FD0DC00D
:101DB0008091B900887F883241F08091740281114E
:101DC00006C092E090937402089581E0089580E047
:101DD0000895109274020895809375021092B900CC
:101DE00084FF05C08CE08093B8000C94E90E88E471
:101DF000FACFCF93DF93FC0123A5222389F0EC01D6
:101E00000E94910E811104C080E0DF91CF9108956E
:101E10008EA1811107C00E94C90E8823A9F31BA6B9
:101E200081E0F3CF80E4F7CF0F931F93CF93DF933D
:101E3000C62FD42F8901633001F138F4613099F055
:101E4000623009F449C0C1E012C0663029F1673040
:101E500091F16530C1F70E94F90E811117C00E94FF
:101E6000C20EC0E004C0FC0186A50E94EC0E8C2FBF
:101E7000DF91CF911F910F910895FC0116A221E0EF
:101E800023A74111E0CF0E94C20EDDCF8D2F0E940B
:101E9000C90E8111D8CFE3CF0E94F90E8823F9F241
:101EA000DD2389F2F80181918F010E94C90E8823F8
:101EB000B1F2D150F5CF0E94F90E882381F2DD23D3
:101EC00011F2F80184910E94C90EC82F882379F27B
:101ED0000F5F1F4FD150F3CFFC0146A321E023A792
:101EE000B2CFDB011496ED91FC9130E020E065E08B
:101EF0000994DB011496ED91FC9130E020E062E062
:101F00000994DB011496ED91FC9130E020E063E050
:101F10000994CF92DF92EF92FF920F931F93CF938A
:101F2000DF938C017B016A0180E0F601C49181118D
:101F300010C081E0CF3F49F04C2FB701C8010E948B
:101F4000710F882309F444C080E0BFEFCB1ADB0A8D
:101F5000ECCF4FEFCF3F89F3CE3FD9F1C03FA0F791
:101F6000C03E38F04C2F4F70B701C8010E94790F66
:101F7000EBCFC03D38F04C2F4F70B701C8010E9425
:101F8000810FE2CFC03CF8F0D7011496ED91FC919F
:101F900030E020E040E064E0C8010995C295C07FD0
:101FA000CE5FD0E0CE010E945D0ED7011496ED9178
:101FB000FC9130E020E041E064E0C8010995CE01E9
:101FC0000E945D0EC1CFC7FDBFCF8C2F90E0F8CF30
:101FD00080E0DF91CF911F910F91FF90EF90DF9004
:101FE000CF900895AF92BF92CF92DF92FF920F935E
:101FF0001F93CF93DF936C018B01F42EE90180E1F5
:10200000481709F47EC0841778F1AAE04A1709F44A
:1020100061C0BFE04B1709F47FC0F8010281138152
:10202000F2E3FF1609F4DDC0FF1508F48EC085E168
:10203000F81609F4DBC0A7E1FA1609F4ECC0B4E124
:10204000FB1265C0D8011696ED91FC911797159675
:102050008C918E0F9F2F911D11928E179F07E1F784
:10206000C8010E94D70C53C0E1E14E1709F451C0DA
:10207000F5E14F13D2CFFB01A280B3804CE750E0D3
:10208000C6010E94890FD50114964C91406BB8018E
:10209000C6010E94710F41E0B801C6010E94790F8C
:1020A000F50126813781D8011496ED91FC91D50177
:1020B00015964C9166E0C601099581111CC080E01F
:1020C000DF91CF911F910F91FF90DF90CF90BF9044
:1020D000AF900895DB011496ED91FC9130E020E083
:1020E00042E061E0C601099544E850E0B801C6014C
:1020F0000E94890F92CF40E0B801C6010E94810F73
:102100008CCF43E750E0B801C6010E94890F81E0FF
:10211000D7CF48E650E0F7CF41E0C6010E94810FDB
:1021200040E0B801C6010E94790F41E8B801C6013C
:102130000E94710F4881B801C6010E94710F40E0F2
:10214000B801C6010E94810FE2CFE6E4FE1609F451
:102150006CC0F7E4FF1609F46DC08BE3F812D7CF1B
:1021600099818B8138E0390F813031F0833011F063
:10217000392F02C0392F985021E0D80113964C9185
:10218000491708F420E041E0391708F040E091E0F9
:10219000F8015281351708F490E0322F342B932345
:1021A00019F4242309F4B3CFFA80D12CC12C843044
:1021B00048F490E0FC01EB5DFE4FC0808F5D9E4FC8
:1021C000DC01DC90F7FE04C0BE01C8010E94AB0C2C
:1021D00088818C0D888389818D0D8983FF0C91F70F
:1021E00096CFBE01C8010E94AB0C91CFC8010E94DE
:1021F000C10C882309F463CFD8011696ED91FC91A8
:10220000179715968C918E0F9F2F911D11928E17F7
:102210009F07E1F77CCF1882F8018281898385814D
:1022200081508A8383818B8372CFD80115968C91DC
:1022300088836DCFF8018181FBCFFC014150460FAF
:1022400093A985A9861738F081E0491740F446170D
:1022500008F080E008954917E0F381E0F8CF089591
:10226000CF93DF9390912E039630A0F090912C03A2
:102270009B3080F4D62FC82F462F682F88EF92E02E
:102280000E941D11882331F06D2F8C2FDF91CF918B
:102290000C947B0DDF91CF9108951F93CF93DF9323
:1022A000C1E0C0930202882399F1D091B800109147
:1022B000BA008091BC008A7B8093BC0060E082E120
:1022C0000E94BD0B60E083E10E94BD0B1092BE0234
:1022D000C093BD021092980261E082E10E94BD0BA2
:1022E00061E083E10E94BD0B8091B9008E7F8093F5
:1022F000B9008091B9008D7F8093B90088E4809304
:10230000B80085E48093BC001093BA00D093B80065
:10231000DF91CF911F9108958F929F92AF92BF92BC
:10232000CF92DF92EF92FF920F931F93CF93DF93A1
:10233000D091E702D13208F0D7C0182FC091E60241
:102340000E943A0C6B017C018091BE0281116BC02E
:1023500082E08093BE021093BD028FEF8093BC0297
:102360001092BB02D093BA02A6ECB2E0EAE9F2E026
:1023700080E0D81391C01092990280919902CC0FFD
:10238000C82BC093990280919802813009F088C0CF
:10239000109298020E943A0C6B017C018091990284
:1023A0008093BB008091C0029091C102A091C202B3
:1023B000B091C302892B8A2B8B2BA1F00E943A0C7F
:1023C0000091C0021091C1022091C2023091C3025B
:1023D0006C197D098E099F09061717072807390709
:1023E00008F442C08091BC0083FDD8CF85EC809377
:1023F000BC000E943A0C6B017C018091BE028230CD
:1024000009F450C08091BC028F3F09F46FC08091E5
:10241000BC02803209F46CC08091BC02803309F4A4
:1024200069C084E026C08091C0029091C102A09151
:10243000C202B091C302892B8A2B8B2B09F484CF63
:102440000E943A0C8090C0029090C102A090C202FB
:10245000B090C3026C197D098E099F0986169706F4
:10246000A806B90608F070CF8091BF020E944D11F6
:1024700085E01092C5021092E7021092C402DF912B
:10248000CF911F910F91FF90EF90DF90CF90BF9071
:10249000AF909F908F9008959D9191938F5F69CF9A
:1024A00085EEA5CF8091C0029091C102A091C20299
:1024B000B091C302892B8A2B8B2B09F49ECF0E94EB
:1024C0003A0C0091C0021091C1022091C2023091D9
:1024D000C3026C197D098E099F0906171707280783
:1024E000390708F08ACFC0CF81E0C3CF80E0C1CFE9
:1024F00082E0BFCF83E0BDCF20912302260F332798
:10250000331F21323105ECF42091BE02FC0190E032
:1025100080E0243069F082E00895A09123022191A7
:10252000AC014D5F5D4FA40FB52FB11D2C930196EB
:10253000861798F380912302680F6093230280E04E
:10254000089581E008950895E091770280917602E0
:10255000E81730F4F0E0E858FD4F808190E00895EE
:102560008FEF9FEF089590917702809176022FEF81
:102570003FEF981748F4E92FF0E0E858FD4F20812D
:1025800030E09F5F90937702C9010895CF92DF9268
:10259000EF92FF920F931F93CF93DF937C01CB01B8
:1025A0008A012091C402222389F0EB016B01C40E41
:1025B000D51ECC15DD0569F06991D701ED91FC912F
:1025C0000190F081E02DC7010995F3CF642F0E949F
:1025D0007C12C801DF91CF911F910F91FF90EF9076
:1025E000DF90CF900895CF93DF931F92CDB7DEB7E2
:1025F00069832091C4022223F9F02091E70220325E
:1026000058F021E030E0FC013383228390E080E049
:102610000F90DF91CF9108958091C502E82FF0E0EF
:10262000EA53FD4F998190838F5F8093C502809319
:10263000E70281E090E0ECCF61E0CE0101960E94DC
:102640007C12F7CF91E09093C40290E49093E6025D
:102650001092C5021092E702682F88EE92E00E9465
:10266000F31281E00C948C118EBD00000DB407FEB6
:10267000FDCF8EB50895CF93DF93C82FD62F60E09E
:102680008AE00E94BD0B80E28C0FC03238F08FE1EF
:102690008C0F833088F0CF3F79F08C2F0E94341359
:1026A000C82F8D2F0E94341361E08AE00E94BD0B79
:1026B0008C2FDF91CF9108958C2F0E943413C82F57
:1026C000F3CFCF93C82F60E08AE00E94BD0B8C2F20
:1026D0000E94341380E00E943413C82F61E08AE026
:1026E0000E94BD0B8C2FCF910895EF92FF920F9314
:1026F0001F93CF93DF93C82FF62EE72ED42F86306B
:1027000019F080F4823080F483E00E946113D2E0FB
:10271000D80F60E08AE00E94BD0B8AE28C0F0E9415
:10272000341302C0873071F00F2D1E2DD15080F46C
:1027300061E08AE0DF91CF911F910F91FF90EF90C0
:102740000C94BD0B60E08AE00E94BD0B80EAE7CFED
:10275000F80181918F010E943413E8CF3F924F928C
:102760005F926F927F928F929F92AF92BF92CF9221
:10277000DF92EF92FF920F931F93CF93DF93EC01C1
:10278000B62EFCAC9BAC6C0124E0C20ED11CE98DD2
:10279000FA8DC6010995882E08851985C8010E9401
:1027A0003E0EE82E888599850E94410E682E81E0B4
:1027B00077247A94E81202C02FE0722E88859985DA
:1027C0000E943A0EE82E888599850E94360EA82E22
:1027D000888599850E94570EE0E6EB1578F40097FE
:1027E00069F0080F191F91E6E92EAB14C0F41C8A9A
:1027F0001F8A188E1D8A1E8A80E09DC08885998553
:102800000E945A0EF0E4FB1538F4009729F0080FE7
:10281000191F81E4E82EE9CF0F5E1F4FE6CFAE14FB
:1028200030F3862D90E0F80124912F3F31F40F5FB3
:102830001F4FAE14E1F2E394F6CFBE106FC088854F
:1028400099850E943E0E98012F5F3F4FF801882323
:1028500019F0823009F04BC084918F8BF9012491DB
:10286000288FF8013396E491EC8BF8013496E491CB
:10287000ED8BF8013596E491EE8B0115110509F405
:10288000BBCF888599850E94410EB82E388C7F2C4D
:1028900073188E89781A780C8FEF830D870D98AD99
:1028A0002AAD271508F443C0891718F4871508F0D6
:1028B00041C06F885D88590C462D652DC6010E9468
:1028C0001D11882309F436C00B0D111DF7E06F0EA2
:1028D000669466946694370C5E0120E2A20EB11CE9
:1028E000862C912C731431F1452C78014DC08491C4
:1028F000982F9F7092509E8B82958F708D8BF901CF
:102900002491822F8F70888F22952F702F8BF80142
:102910003296E491E295EF70EC8BAFCF3296E49172
:10292000E721E80FF92FF11D0E0F1F1F82CF891726
:1029300008F0BCCF8C899BAD890F8BAF81E090E014
:10294000DF91CF911F910F91FF90EF90DF90CF908B
:10295000BF90AF909F908F907F906F905F904F90BF
:102960003F900895F70184916E817F8148A279A2FA
:102970001BA28AA395014BE3C6010E94DE0CFFEF68
:10298000EF1AFF0A28E0420E8E2D801B861550F3A9
:10299000080D191D7394A6CF089590E080E0089566
:1029A0008F929F92AF92BF920F931F93CF93DF931B
:1029B000CDB7DEB7A1970FB6F894DEBF0FBECDBF7F
:1029C00019A2423008F44AE08E010F5D1F4F842E99
:1029D000912CB12CA12CA50194010E949D20E62FE1
:1029E000B901CA01EA3044F5E05DD801EE938D01EA
:1029F000232B242B252B79F790E080E0109769F0AA
:102A0000FD0101900020E9F73197AF014A1B5B0BF4
:102A1000BD0184EF92E00E94900BA1960FB6F8944E
:102A2000DEBF0FBECDBFDF91CF911F910F91BF9041
:102A3000AF909F908F900895E95CD7CFFC010190F3
:102A40000020E9F73197AF01481B590BBC0184EF17
:102A500092E00C94900BCF92DF92EF92FF92CF9383
:102A6000DF936C01990FEE08FF08F7FE19C06DE2C5
:102A700084EF92E00E94AE13EC0166277727CB012A
:102A80006C197D098E099F094AE00E94D0148C0FB1
:102A90009D1FDF91CF91FF90EF90DF90CF90089531
:102AA0004AE0C701B601DF91CF91FF90EF90DF9030
:102AB000CF900C94D0148F929F92AF92BF92CF92EE
:102AC000DF92EF92FF921F93CF93DF930E943A0C15
:102AD0006B017C018091BE02811165C081E0809311
:102AE000BE028093BD029FEF9093BC021092BB0286
:102AF00092E09093BA028093990280919902806843
:102B00008093990280919802813009F089C01092D7
:102B100098020E943A0C6B017C018091990280938B
:102B2000BB008091C0029091C102A091C202B091FD
:102B3000C302892B8A2B8B2BA1F00E943A0C809028
:102B4000C0029090C102A090C202B090C3026C1962
:102B50007D098E099F0986169706A806B90608F40E
:102B600043C08091BC0083FDD8CF85EC8093BC002E
:102B70000E943A0C6B017C018091BE02813009F405
:102B800051C08091BB02D3E0833010F4D091BB02DE
:102B9000AAE9B2E0E8E7F2E080E08D1751F19D91FB
:102BA00091938F5FFACF8091C0029091C102A09162
:102BB000C202B091C302892B8A2B8B2B09F48ACFD6
:102BC0000E943A0C8090C0029090C102A090C20274
:102BD000B090C3026C197D098E099F09861697066D
:102BE000A806B90608F076CF8091BF020E944D1169
:102BF000D0E010927702D093760280917702D817B6
:102C000099F188EE92E00E94B312C82F88EE92E00C
:102C10000E94B312182F88EE92E00E94B312EDCFFB
:102C200085EEA4CF8091C0029091C102A091C20212
:102C3000B091C302892B8A2B8B2B09F49DCF0E9464
:102C40003A0C8090C0029090C102A090C202B09055
:102C5000C3026C197D098E099F0986169706A8067E
:102C6000B90608F089CFC0CF6C2F70E090E080E00B
:102C7000982F872F762F6627610F711D811D911D5B
:102C8000DF91CF911F91FF90EF90DF90CF90BF9099
:102C9000AF909F908F90089585ED8093BC008091B8
:102CA000C0029091C102A091C202B091C3020796E6
:102CB000A11DB11D23E0B695A795979587952A95F7
:102CC000D1F72091BC0024FD03C01092BE020895EC
:102CD0004091C0025091C1026091C2027091C30242
:102CE000452B462B472B69F30097A105B10541F011
:102CF00025E32A95F1F700000197A109B109E1CF79
:102D00008091BF020C944D111F920F920FB60F923B
:102D100011242F933F938F939F93AF93BF938091F1
:102D2000470290914802A0914902B0914A02309125
:102D3000460223E0230F2D3758F50196A11DB11D42
:102D4000209346028093470290934802A093490241
:102D5000B0934A0280914B0290914C02A0914D0297
:102D6000B0914E020196A11DB11D80934B0290932C
:102D70004C02A0934D02B0934E02BF91AF919F9130
:102D80008F913F912F910F900FBE0F901F9018952C
:102D900026E8230F0296A11DB11DD2CF1F920F92DC
:102DA0000FB60F9211242F933F934F935F936F931E
:102DB0007F938F939F93AF93BF93EF93FF938091F4
:102DC000B900887F803609F44AC0F0F5883209F4EA
:102DD000A5C018F5803109F499C0B8F4882309F426
:102DE000F5C0883009F492C0FF91EF91BF91AF9187
:102DF0009F918F917F916F915F914F913F912F9113
:102E00000F900FBE0F901F901895883109F486C05F
:102E1000803251F78093BC0214C0803409F49BC007
:102E200040F48033B9F38833F9F68093BC0285EC23
:102E3000AEC0803509F483C0883509F494C0883465
:102E400099F60E944C16D0CF883909F48AC038F51B
:102E5000883729F050F4883611F0803729F683E05E
:102E60008093BE021092450255C0883809F479C09B
:102E7000803919F0803809F0B7CF8091450280324F
:102E800008F06FC0E091450281E08E0F809345020B
:102E90008091BB00F0E0EB5DFD4F80833BC0803B49
:102EA00039F0D0F4803A09F477C0883A09F09CCF21
:102EB00084E08093BE021092240210922302F0E07C
:102EC000E0E009958091230281110FC081E0809399
:102ED00023021092030209C0803C09F4A8CF883C69
:102EE00009F4A5CF883B09F07FCFE091240281E06F
:102EF0008E0F80932402F0E0ED5FFD4F8081809380
:102F0000BB00909124028091230229C080919902F4
:102F10008093BB0085EC8093BC0066CF9091BB0290
:102F20008091BA02981758F5E091BB0281E08E0FAC
:102F30008093BB02F0E0E656FD4F8081E9CFE0913F
:102F4000BB0281E08E0F8093BB028091BB00F0E05A
:102F5000E656FD4F80839091BB028091BA0298178C
:102F6000C8F285E8D8CFE091BB0281E08E0F809354
:102F7000BB028091BB00F0E0E656FD4F808380915C
:102F8000BD0281115ECF81E08093980284EA809334
:102F9000BC001092BE0228CF85EC8093BC0010923A
:102FA000BE0280914502803230F4E0914502F0E0AB
:102FB000EB5DFD4F10826091450270E085E292E08A
:102FC000F0E0E0E00995109245020ECF1092BC02AD
:102FD00038CF1092EB021092EA0288EE93E0A0E064
:102FE000B0E08093EC029093ED02A093EE02B093D8
:102FF000EF028DE291E09093E9028093E80260E0B5
:1030000082E00E94090CE2EFF4E0E491E0933203E5
:10301000EEEDF4E0E491F0E0EE0FFF1FEE52FB4F17
:1030200085919491909334038093330310923D03E0
:1030300010923F0310923E0310923C0310923B0308
:1030400010923A031092390310923803109237030A
:1030500010923603109235031092F7021092F60286
:103060008FE391E09093F5028093F40210922F0386
:1030700010923003109231031092FD021092FC0264
:103080001092FF021092FE021092010381E08093E1
:10309000000382E28093020310920703109206035A
:1030A000EBE1F3E08FEF819393E0E932F907D9F791
:1030B00081E08093180329E43BE030930E032093D2
:1030C0000D0380930F03109210031092110380E4FC
:1030D000809312031092130388E49BE090932A03D9
:1030E0008093290386E191E09093FB028093FA029A
:1030F00082E1809326030E94E20C8FE391E090939B
:10310000F5028093F4020895CF93DF93CDB7DEB735
:1031100069970FB6F894DEBF0FBECDBF789484B523
:10312000826084BD84B5816084BD85B5826085BDC3
:1031300085B5816085BD80916E00816080936E0051
:103140001092810080918100826080938100809143
:1031500081008160809381008091800081608093F4
:1031600080008091B10084608093B1008091B000B4
:1031700081608093B00080917A00846080937A00AF
:1031800080917A00826080937A0080917A008160D9
:1031900080937A0080917A00806880937A00109200
:1031A000C1001FB7F89480914F02811127C0E6EE4D
:1031B000F4E08491EAEFF4E09491E82FF0E0EE0F70
:1031C000FF1FE853FF4FA591B491EC91E92321F43F
:1031D00061E08AE00E94BD0B61E08AE00E94090C78
:1031E0008CB580618CBD8CB580648CBD61E08DE058
:1031F0000E94090C61E08BE00E94090C80914F0253
:103200008F5F80934F021FBF61E08AE00E94090C2C
:1032100061E08AE00E94BD0B61E089E00E94090C38
:1032200060E089E00E94BD0B85E0ECE1F1E09E01E9
:103230002F5F3F4F5901D90101900D928A95E1F717
:1032400068EC70E080E090E00E945F0C60E787E04F
:103250000E943B1360E082E00E943B1360E081E04B
:103260000E943B1360E181E10E943B1380E00E94D9
:103270006113682F6C6080E00E943B1363E083E081
:103280000E943B1340E0B50186E00E94751380E088
:103290000E946113682F6E7F80E00E943B1364E6FA
:1032A00085E00E943B1380E00E946113682F6260FA
:1032B00080E00E943B1362E070E080E090E00E94BA
:1032C0005F0C789464EF71E080E090E00E945F0C06
:1032D000A9E42A2EABE03A2E64E670E080E090E0AC
:1032E0000E945F0C6AE070E080E090E00E945F0C5A
:1032F00083EE90E00E9422130E945B150E94671FDC
:1033000020E030E040E857E30E94F81F22E538EB68
:103310004FE253E40E94F81F26E636E64BE352E400
:103320000E94501E2DEC3CEC4CE85FE30E94501EC6
:103330006B017C0164E670E080E090E00E945F0C2D
:1033400085EE90E00E9422130E945B150E94671F89
:1033500020E030E040E857E30E94F81F20E030E032
:103360004AEF52E40E94F81F20E030E040EC50E4C5
:103370000E94501E2B013C01C701B6010E942F1F65
:103380006A8B7B8B8C8B9D8B0A891B891093130115
:103390000093120120E030E040E251E4C701B601A1
:1033A0000E94F81F6E8B7F8B888F998F8AE0809F99
:1033B000B001819F700D1124072E000C880B990B12
:1033C0000E94671F9B01AC016E897F89888D998D52
:1033D0000E94501E6B017C0120E030E0A9010E9498
:1033E000F31F18160CF0CAC2C701B6010E942F1FA6
:1033F0007093110160931001C301B2010E942F1F4D
:103400006B0170930F0160930E0120E030E040E209
:1034100051E4C301B2010E94F81F2B013C018AE074
:103420008C9DB0018D9D700D1124072E000C880B12
:10343000990B0E94671F9B01AC01C301B2010E945E
:10344000501E0E942F1F70930D0160930C0117FFF7
:1034500004C010921501109214018EE480937C0038
:1034600020E031E080E090E0DC0140917A00406CA7
:1034700040937A0040917A0046FDFCCF409178005D
:1034800050917900840F951FA11DB11D2150310964
:1034900061F720917A002F7720937A00BC01CD014B
:1034A000F4E09595879577956795FA95D1F7072E6E
:1034B000000C880B990B0E94671F9B01AC0161E611
:1034C00073E583ED99E40E94BD1E0E942F1FCB017E
:1034D00064E670E00E94892070930B0160930A01FA
:1034E0009093090180930801209172023091730238
:1034F000232B09F0FDC044E6469F9001479F300D05
:103500001124820F931F40911201509113012AE060
:10351000249F6001259FD00C1124409110015091EF
:103520001101C40ED51E40910E0150910F01249F30
:103530007001259FF00C112420910C0130910D0198
:10354000E20EF31E9E01225F3F4F39018436910542
:103550000CF018C29F938F9388E491E09F938F9310
:103560007F926F920E94E0200F900F900F900F902B
:103570000F900F901F9288E38F93E9E48E2EE1E085
:103580009E2E9F928F92BF92AF920E94E0200F904A
:103590000F900F900F900F900F908E01065F1F4FAE
:1035A00034E6C316D1040CF0F2C1DF92CF9288E466
:1035B00091E09F938F931F930F930E94E0200F90B1
:1035C0000F900F900F900F900F908AE0C816D104C3
:1035D00084F4DF92CF9287E491E09F938F931F93BF
:1035E0000F930E94E0200F900F900F900F900F907C
:1035F0000F90FE0136966F01F4E6EF16F1040CF021
:10360000CBC1FF92EF9288E491E09F938F93DF927A
:10361000CF920E94E0200F900F900F900F900F908C
:103620000F902AE0E216F10484F4FF92EF9287E40F
:1036300091E09F938F93DF92CF920E94E0200F90B2
:103640000F900F900F900F900F9080911401909118
:103650001501892B09F0A5C1BF92AF92DF92CF92DD
:103660007F926F921F930F938CE491E09F938F93BF
:1036700080E592E09F938F930E94E0200FB6F8942C
:10368000DEBF0FBECDBF60E572E081E692E00E9432
:10369000D92040E161E672E087E00E94751361E0A5
:1036A00089E00E94BD0B61E070E080E090E00E9444
:1036B0005F0C60E089E00E94BD0B60E08FEF0E942C
:1036C0003B1385FFFACF60E287E00E943B1311E0D5
:1036D0001093C4028CE38093E6021092C50210920C
:1036E000E70281E00E948C11811166C11093710282
:1036F000809172029091730201969093730280936D
:10370000720280917102882309F4BEC20E94480DA2
:103710003AE0832E4BE3442E58E0552E6DE0962E72
:1037200074E6672E80917202909173020A970CF0F2
:1037300090C280912C03803478F440E860E088EFF8
:1037400092E00E941D1192EDE92E90E0F92EC12C1D
:1037500022E0722E811157C18091FC029091FD02EE
:10376000825B994061F022EB39E03093FD022093B7
:10377000FC020E944B0B30920E0320920D038092AC
:103780002F0334E2309330038AE691E00E941E1545
:103790008091140190911501892B09F038C18DE7B2
:1037A00091E00E941E1580911201909113010E94D8
:1037B0002B158FE691E00E941E15809110019091CB
:1037C00011010A9724F481E791E00E941E1580916F
:1037D0001001909111010E942B1580E891E00E9448
:1037E0001E1580922F034092300383E791E00E94E0
:1037F0001E1580910E0190910F010E942B158FE6EE
:1038000091E00E941E1580910C0190910D010A9784
:1038100024F481E791E00E941E1580910C019091A3
:103820000D010E942B1586E791E00E941E158091E4
:10383000FC029091FD028450954061F024E035E057
:103840003093FD022093FC020E944B0B30920E033A
:1038500020920D0350922F039092300380910A0121
:1038600090910B010E942B158FE691E00E941E158E
:1038700080910801909109010A9724F481E791E071
:103880000E941E1580910801909109010E942B153C
:1038900088E791E00E941E1580910A0190910B012A
:1038A000689E8001699E100D1124809108019091FD
:1038B0000901080F191F61E08CE70E9430110139DE
:1038C00031E0130784F063E08AE70E94301163E07F
:1038D00086E70E94301163E082E70E94301163E0C6
:1038E0008EE60E943011C8018D579140449760F4D4
:1038F00063E08AE70E94301163E086E70E9430119E
:1039000063E082E70E943011C801895691404497D4
:1039100040F463E08AE70E94301163E086E70E948A
:1039200030110B5411400E31110520F463E08AE789
:103930000E94301182E380932F03909230038AE734
:1039400091E00E941E158091720290917302EAE04C
:10395000F0E0E81BF90BCF010E942B158FE791E0F7
:103960000E941E150E94A30D8111DCCE80E090E024
:10397000892B09F4B1CC0E940000AECCC701B6017E
:10398000905834CD9F938F9389E491E0E7CDDF92F7
:10399000CF929F928F9223CEFF92EF9289E491E093
:1039A00048CEBF92AF92DF92CF927F926F921F93D9
:1039B0000F938BE591E05ACE1092710299CEF801E7
:1039C00084916091FA027091FB02D0921403C0922C
:1039D0001503709217038093160324E133E04BE341
:1039E00088EF92E00E94DE0C0F5F1F4FF8E0DF0EC1
:1039F00027E8D212E4CF30E1E30EF11CC39480E457
:103A0000C81609F4A9CE870187E0D82ED8CF8DE655
:103A100091E0C7CE0E94480D20E24FE760E280E0CF
:103A20000E94DD0D0E94A30D8111F6CF0E94480D6A
:103A300020E24FE760E280E00E94DD0D0E94A30DCE
:103A40008111F6CF0E94480D20E24BE660E284E14E
:103A50000E94DD0D0E94A30D8111F6CF0E94480D3A
:103A600020E24BE660E284E10E94DD0D0E94A30D9E
:103A70008111F6CF0E94480D20E241E660E28EE11E
:103A80000E94DD0D0E94A30D8111F6CF0E94480D0A
:103A900020E241E660E28EE10E94DD0D0E94A30D6E
:103AA0008111F6CF0E94480D20E247E560E288E2EE
:103AB0000E94DD0D0E94A30D8111F6CF0E94480DDA
:103AC00020E247E560E288E20E94DD0D0E94A30D3E
:103AD0008111F6CF0E94480D20E242E560E28DE2BE
:103AE0000E94DD0D0E94A30D8111F6CF0E94480DAA
:103AF00020E242E560E28DE20E94DD0D0E94A30D0E
:103B00008111F6CF0E94480D20E24DE460E282E38D
:103B10000E94DD0D0E94A30D8111F6CF0E94480D79
:103B200020E24DE460E282E30E94DD0D0E94A30DDD
:103B30008111F6CF0E94480D20E248E460E287E35D
:103B40000E94DD0D0E94A30D8111F6CF0E94480D49
:103B500020E248E460E287E30E94DD0D0E94A30DAD
:103B60008111F6CF0E94480D20E245E460E28AE32D
:103B70000E94DD0D0E94A30D8111F6CF0E94480D19
:103B800020E245E460E28AE30E94DD0D0E94A30D7D
:103B90008111F6CF0E94480D20E242E460E28DE3FD
:103BA0000E94DD0D0E94A30D8111F6CF0E94480DE9
:103BB00020E242E460E28DE30E94DD0D0E94A30D4D
:103BC0008111F6CF0E94480D20E241E460E28EE3CD
:103BD0000E94DD0D0E94A30D8111F6CF0E94480DB9
:103BE00020E241E460E28EE30E94DD0D0E94A30D1D
:103BF0008111F6CF0E94480D20E240E460E28FE39D
:103C00000E94DD0D0E94A30D8111F6CF0E94480D88
:103C100020E240E460E28FE30E94DD0D0E94A30DEC
:103C20008111F6CF6091FA027091FB0230E020E042
:103C300040E188EF92E00E94DE0C83B7817F8460D0
:103C400083BF83B7816083BF889583B78E7F83BF2F
:103C500089CE02E010E00E94480D21E24FE761E2C8
:103C600080E00E94DD0D2FE14FE76FE180E00E94D0
:103C7000DD0D0E94A30D8111F0CF0130110509F473
:103C8000C9CE01E010E0E7CF83B7817F846083BFB6
:103C900083B7816083BF889583B78E7F83BF66CEED
:103CA0005058BB27AA270E94681E0C94B91F0E9477
:103CB000AB1F38F00E94B21F20F039F49F3F19F477
:103CC00026F40C94A81F0EF4E095E7FB0C94A21FB9
:103CD000E92F0E94CA1F58F3BA17620773078407B7
:103CE000950720F079F4A6F50C94EC1F0EF4E095FE
:103CF0000B2EBA2FA02D0B01B90190010C01CA01A6
:103D0000A0011124FF27591B99F0593F50F4503E50
:103D100068F11A16F040A22F232F342F4427585F42
:103D2000F3CF469537952795A795F0405395C9F75A
:103D30007EF41F16BA0B620B730B840BBAF0915012
:103D4000A1F0FF0FBB1F661F771F881FC2F70EC0B1
:103D5000BA0F621F731F841F48F487957795679584
:103D6000B795F7959E3F08F0B0CF9395880F08F070
:103D70009927EE0F9795879508950E94D11E0C9470
:103D8000B91F0E94B21F58F00E94AB1F40F029F4E7
:103D90005F3F29F00C94A21F51110C94ED1F0C945D
:103DA000A81F0E94CA1F68F39923B1F3552391F30A
:103DB000951B550BBB27AA2762177307840738F09A
:103DC0009F5F5F4F220F331F441FAA1FA9F335D0F7
:103DD0000E2E3AF0E0E832D091505040E695001CAB
:103DE000CAF72BD0FE2F29D0660F771F881FBB1F65
:103DF000261737074807AB07B0E809F0BB0B802D43
:103E0000BF01FF2793585F4F3AF09E3F510578F06E
:103E10000C94A21F0C94ED1F5F3FE4F3983ED4F383
:103E2000869577956795B795F7959F5FC9F7880F42
:103E3000911D9695879597F90895E1E0660F771F94
:103E4000881FBB1F621773078407BA0720F0621B25
:103E5000730B840BBA0BEE1F88F7E09508950E9450
:103E6000361F6894B1110C94ED1F08950E94D21F63
:103E700088F09F5798F0B92F9927B751B0F0E1F02B
:103E8000660F771F881F991F1AF0BA95C9F714C0DB
:103E9000B13091F00E94EC1FB1E008950C94EC1F3A
:103EA000672F782F8827B85F39F0B93FCCF3869514
:103EB00077956795B395D9F73EF490958095709571
:103EC00061957F4F8F4F9F4F0895E89409C097FBEE
:103ED0003EF490958095709561957F4F8F4F9F4FE1
:103EE0009923A9F0F92F96E9BB279395F695879525
:103EF00077956795B795F111F8CFFAF4BB0F11F4E8
:103F000060FF1BC06F5F7F4F8F4F9F4F16C088238E
:103F100011F096E911C0772321F09EE8872F762FC4
:103F200005C0662371F096E8862F70E060E02AF005
:103F30009A95660F771F881FDAF7880F96958795F1
:103F400097F9089597F99F6780E870E060E0089519
:103F50009FEF80EC089500240A94161617061806A1
:103F60000906089500240A9412161306140605067D
:103F70000895092E0394000C11F4882352F0BB0F0E
:103F800040F4BF2B11F460FF04C06F5F7F4F8F4F71
:103F90009F4F089557FD9058440F551F59F05F3FAC
:103FA00071F04795880F97FB991F61F09F3F79F05B
:103FB00087950895121613061406551FF2CF4695DD
:103FC000F1DF08C0161617061806991FF1CF86955F
:103FD0007105610508940895E894BB276627772743
:103FE000CB0197F908950E94652008F48FEF08959A
:103FF0000E940B200C94B91F0E94AB1F38F00E9446
:10400000B21F20F0952311F00C94A21F0C94A81F4E
:1040100011240C94ED1F0E94CA1F70F3959FC1F3E9
:10402000950F50E0551F629FF001729FBB27F00D66
:10403000B11D639FAA27F00DB11DAA1F649F6627BB
:10404000B00DA11D661F829F2227B00DA11D621F0A
:10405000739FB00DA11D621F839FA00D611D221FC4
:10406000749F3327A00D611D231F849F600D211DA8
:10407000822F762F6A2F11249F5750409AF0F1F02B
:1040800088234AF0EE0FFF1FBB1F661F771F881F94
:1040900091505040A9F79E3F510580F00C94A21F0B
:1040A0000C94ED1F5F3FE4F3983ED4F3869577952B
:1040B0006795B795F795E7959F5FC1F7FE2B880F3A
:1040C000911D9695879597F90895990F0008550FBA
:1040D000AA0BE0E8FEEF16161706E807F907C0F08E
:1040E00012161306E407F50798F0621B730B840B96
:1040F000950B39F40A2661F0232B242B252B21F470
:1041000008950A2609F4A140A6958FEF811D811D0F
:10411000089597FB072E16F4009407D077FD09D079
:104120000E94BF2007FC05D03EF4909581959F4FDB
:104130000895709561957F4F0895A1E21A2EAA1BEC
:10414000BB1BFD010DC0AA1FBB1FEE1FFF1FA21747
:10415000B307E407F50720F0A21BB30BE40BF50B44
:10416000661F771F881F991F1A9469F760957095CD
:10417000809590959B01AC01BD01CF010895AA1BCC
:10418000BB1B51E107C0AA1FBB1FA617B70710F042
:10419000A61BB70B881F991F5A95A9F78095909574
:1041A000BC01CD010895EE0FFF1F0590F491E02DA5
:1041B0000994FB01DC0101900D920020E1F70895C4
:1041C000AEE0B0E0E6EEF0E20C948F230D891E899C
:1041D00086E08C831A8309838FEF9FE79E838D830C
:1041E000AE01475E5F4F6F89788DCE0101960E94C8
:1041F00003212F813885020F131FF80110822E969C
:10420000E4E00C94AB23ABE0B0E0E9E0F1E20C9425
:1042100081237C013B018A01FC0117821682838184
:1042200081FFC8C1CE0101965C01F7019381F301C2
:1042300093FD859193FF81913F01882309F453C138
:10424000853239F493FD859193FF81913F01853249
:1042500029F4B70190E00E94F322E7CF912C212CA2
:10426000312CFFE1F31538F08B3211F190F48032EC
:1042700009F1833229F137FC3CC020ED280F2A30A8
:1042800050F536FE20C08AE0989E200D1124922E13
:1042900006C08D3291F0803371F7689430F8F301E5
:1042A00093FD859193FF81913F018111DACF21C068
:1042B000689431F8689432F8F2CF689433F8EFCF0D
:1042C000689434F8ECCFEAE02E9E200D1124222EC3
:1042D000689435F8E4CF8E3229F436FC04C1689432
:1042E00036F8DDCF8C3619F4689437F8D8CF883695
:1042F000B1F2982F9F7D95549330E0F08336A1F171
:104300008337C1F1833509F063C02801F2E04F0E15
:10431000511CF801C080D180692D70E036FC02C0CC
:104320006FEF7FEFC6010E94DD224C01689437F8E1
:1043300082010AC00C5F1F4FFFE3F9838824839436
:10434000912C6501E89437F833FE2DC0522C81146E
:10435000910471F5552009F468CFB70180E290E02F
:104360000E94F3225A94F6CFF801808189830E5F70
:104370001F4FE4CF2801F2E04F0E511CF801C0801E
:10438000D180692D70E036FC02C06FEF7FEFC6016F
:104390000E94E8224C018201D5CFB70180E290E073
:1043A0000E94F3222A942814190409F0B0F7CECF02
:1043B000F60137FC859137FE81916F01B70190E0DE
:1043C0000E94F32251105A94F1E08F1A9108BFCF46
:1043D000843619F0893609F077C0F80137FE6BC0D2
:1043E00060817181828193810C5F1F4FF32DFF7675
:1043F0003F2E97FF09C090958095709561957F4FEE
:104400008F4F9F4F689437F82AE030E0A5010E9453
:104410002323C82ECA188C2C432C36FE0CC0E894DB
:1044200040F8C91440F434FE05C032FC03C0F32D3B
:10443000FE7E4F2E892C44FE95C0FE01EC0DF11D31
:104440008081803309F087C0242D297E422E842D5F
:104450008870582E43FC95C040FE8FC09C2C82145F
:1044600018F42C0C922C981844FE91C0B70180E3EC
:1044700090E00E94F32242FE09C088E790E041FEEE
:1044800002C088E590E0B7010E94F322C91408F445
:104490008AC0CA94D12C9FEFC91AD90ACA0CDB1C56
:1044A000F60182916F01B70190E00E94F322AC14F3
:1044B000BD04B1F74FCF60817181072E000C880BCE
:1044C000990B0E5F1F4F92CFD32CE894D4F82AE0BB
:1044D00030E0853739F1232D297FD22E8F3601F137
:1044E00048F48835A9F0F701868197812B96E2E19F
:1044F0000C949D23803749F08837A9F7D4FE02C079
:104500006894D2F820E130E00DC06894D4F8F6CF7A
:1045100034FE03C0822F8660D82E20E132E002C034
:1045200028E030E0F801D7FE0FC060817181828100
:1045300093810C5F1F4FA5010E942323C82ECA1828
:104540003D2CE89437F867CF6081718190E080E07E
:104550000E5F1F4FF0CF42FC02C0839478CF83944C
:10456000839475CF842D867809F471CFF6CFB70187
:1045700080E290E00E94F32283948214C0F3512CD5
:1045800073CF522C5818821408F46ECFF8CF842DB4
:10459000867809F47BCF8BE241FE80E247FC8DE216
:1045A000B70190E071CFB70180E390E00E94F32261
:1045B0009A946CCF8FEF9FEF99CFFC0105906150DB
:1045C00070400110D8F7809590958E0F9F1F089529
:1045D000FC016150704001900110D8F780959095D2
:1045E0008E0F9F1F08950F931F93CF93DF93182F64
:1045F000092FEB018B8181FD09C01FEF0FEF812F88
:10460000902FDF91CF911F910F91089582FF14C0D9
:104610002E813F818C819D81281739073CF4E881E8
:10462000F981CF0101969983888310838E819F81C0
:1046300001969F838E83E3CFE885F985812F0995C5
:10464000892BA1F3DACFFA01AA27283051F12031C2
:1046500081F1E8946F936E7F6E5F7F4F8F4F9F4F16
:10466000AF4FB1E03ED0B4E03CD0670F781F891F58
:104670009A1FA11D680F791F8A1F911DA11D6A0F26
:10468000711D811D911DA11D20D009F468943F91D9
:104690002AE0269F11243019305D3193DEF6CF01D8
:1046A0000895462F4770405D4193B3E00FD0C9F79E
:1046B000F6CF462F4F70405D4A3318F0495D31FD0B
:1046C0004052419302D0A9F7EACFB4E0A69597955E
:1046D000879577956795BA95C9F700976105710534
:1046E00008959B01AC010A2E06945795479537957E
:1046F0002795BA95C9F7620F731F841F951FA01DD8
:1047000008952F923F924F925F926F927F928F9275
:104710009F92AF92BF92CF92DF92EF92FF920F9350
:104720001F93CF93DF93CDB7DEB7CA1BDB0B0FB65A
:10473000F894DEBF0FBECDBF09942A883988488817
:104740005F846E847D848C849B84AA84B984C884AD
:10475000DF80EE80FD800C811B81AA81B981CE0FA4
:10476000D11D0FB6F894DEBF0FBECDBFED01089589
:04477000F894FFCFEB
:1047740008400000008082010800050006004B008C
:10478400030019000100F20F0001140FE2E423E416
:1047940002000100FF0100FF0000000000F312C648
:1047A40012CD14A312890BB312A41200000000AEA0
:1047B40013900BCD14CC14303025640074312D25A6
:1047C400736325737625736825730074312B257301
:1047D40063257376257368257300543D002B002EE2
:1047E400003000483D00250076004F46462D00204D
:0247F400630060
:00000001FF
